:020000040000FA
:1000000000000730990083169F01CD3085008113D1
:10001000831215141515A001900105168B10851675
:100020000230AB2085120230AB208B1C0E2805124B
:100030002030051C1A30A1004E30051C4130A200B2
:10004000752090200430A0077520902003193928CE
:10005000031839280430A00703182F2824288316F2
:100060009B010301992083169B0A03019920051621
:10007000382883167C309B002608992083169B0A1B
:100080002508992083169B0A2408992083169B0A29
:1000900023089920A509A609A50A0319A60A0000A4
:1000A0002508A302031CA4032608A402A41B5E289F
:1000B000A00383167B309B000030992083169B01A0
:1000C00034309920200883169B0A992085168514C0
:1000D00070200000000000008510702000006728DC
:1000E0001730FF3E031D712808002308A5002408CF
:1000F000A60020088316900083120301013E031D11
:100100007E288E018F018B108B1C842810148B107D
:100110008B1C882810100E08A3000F08A4000800EC
:100120002108A302031CA4032208A4022408230418
:10013000080083169A001C1555309D00AA309D00BA
:100140009C1483128C1FA2288C130800A700B120D6
:10015000A70BA7280800A8006430A620A80BAC288D
:100160000800C6300000FF3E031DB228000000005A
:100170000000080043346F347034793472346934C9
:1001800067346834743420345034653474346534DE
:1001900020344734723469346634663469347434D4
:1001A00068347334203428344334293420343234CE
:1001B0003034303437342034313432344634363409
:1001C000323437342F3436343734353420344F34E6
:1001D00053344334433441344C3420347234653422
:1001E000633461346C34693462347234613474342D
:1001F00069346F346E34203431342E343034333437
:020200002034A8
:02400E00A43FCD
:00000001FF
